:100000005CC16BC1A7C269C168C167C1A5C265C136
:1000100064C163C103C462C160C15FC168C4C9C4B3
:100020005CC15BC15AC1000000000000000000007C
:1000300000000000000000000000000000000000C0
:1000400000000000000000000000000000000708A1
:100050000A0B0D0F111315171A1C1F2224272A2D06
:100060003034373A3E4145484C5054575B5F6367E4
:100070006B6F73777B7F83878B8F93979B9FA3A7F0
:10008000ABAFB2B6BABDC1C4C8CBCED1D4D7DADD1E
:10009000E0E2E5E7EAECEEF0F2F3F5F7F8F9FAFB67
:1000A000FCFDFEFEFFFFFFFFFFFFFEFEFDFCFBFA77
:1000B000F9F8F7F5F3F2F0EEECEAE7E5E2E0DDDA85
:1000C000D7D4D1CECBC8C4C1BDBAB6B2AFABA7A34B
:1000D0009F9B97938F8B87837F7B77736F6B676310
:1000E0005F5B5754504C4845413E3A3734302D2AD7
:1000F0002724221F1C1A171513110F0D0B0A0807AE
:10010000000306090C0F1215181B1E212326292C8B
:100110002F3134373A3C3F414446494B4D505254BD
:1001200056585A5C5E6062646567696A6C6D6E7091
:10013000717273747576767778787979797A7A7A54
:100140007A7A7A7A7979797878777676757473723B
:1001500071706E6D6C6A6967656462605E5C5A5846
:10016000565452504D4B494644413F3C3A37343146
:100170002F2C292623211E1B1815120F0C090603EC
:10018000808386898C8F9295989B9EA1A3A6A9AC0B
:10019000AFB1B4B7BABCBFC1C4C6C9CBCDD0D2D43D
:1001A000D6D8DADCDEE0E2E4E5E7E9EAECEDEEF011
:1001B000F1F2F3F4F5F6F6F7F8F8F9F9F9FAFAFAD4
:1001C000FAFAFAFAF9F9F9F8F8F7F6F6F5F4F3F2BB
:1001D000F1F0EEEDECEAE9E7E5E4E2E0DEDCDAD8C6
:1001E000D6D4D2D0CDCBC9C6C4C1BFBCBAB7B4B1C6
:1001F000AFACA9A6A3A19E9B9895928F8C8986836C
:100200004572776172746520434C495000416E72AB
:100210007566004B6C696E0B656C6E200041620B5D
:1002200065686F62656E004175660B656C650B7481
:100230000020416E727566006F686E65204E756DA8
:100240006D657200756E7665726D697474656C7437
:1002500000756E7465726472F5636B74006F686E1E
:1002600065205568727A65697400FC1314166E185F
:10027000FB1AAA224E26592AD32E150A11111F1134
:1002800011001100111111110E000E11111E11118A
:100290001E0000000F11110F010E020006020202E3
:1002A000120C00001111110F010E000000000000DF
:1002B0000000000000000000000011241FBECFE578
:1002C000D2E0DEBFCDBF21E0A0E6B0E001C01D92CC
:1002D000A032B207E1F734D470C592CEC29A0F9221
:1002E0001F926F937F93CF93DF93EF93FF930FB69C
:1002F0000F9265B167FF04C061950AF46A95606862
:10030000D0E0CDE7F0E0E881E39509F4EEE4E9938D
:100310007491112460FD170E1794889461FD170ED7
:100320001794889462FD170E1794889463FD170E36
:100330001794889464FD170E1794889465FD170E22
:100340001794889466FD170E1794889467FD089497
:100350001794612D062E112407FE04C07FE707269F
:1003600003941A947881700D79937881711D799333
:1003700011247FE7762360FD170E1694079461FD24
:10038000170E1694079462FD170E1694079463FDDA
:10039000170E1694079464FD170E1694079465FDC6
:1003A000170E1694079466FD170E1694079416946C
:1003B00007947881700D79937881711D7993002469
:1003C00017FC0A947881701D7993F1E009901990D7
:1003D000E881E00DE993E881E11DE993749111242E
:1003E000062E07267F7760FD170E1694079461FD91
:1003F000170E1694079462FD170E1694079463FD6A
:10040000170E1694079464FD170E1694079465FD55
:10041000170E1694079466FD170E169407941694FB
:10042000079420F41094019408F013947881700DCF
:1004300079937881711D7993002417FC0A9478814F
:10044000701D7993E05474911124062E07267F774E
:1004500060FD170E1694079461FD170E169407940D
:1004600062FD170E1694079463FD170E16940794F9
:1004700064FD170E1694079465FD170E16940794E5
:1004800066FD170E169407941694079420F41094A2
:10049000019408F013947881700D79937881711D1F
:1004A0007993002417FC0A947881701D799373ED79
:1004B000C7138CCFD0E0CDE779917F3F09F03EC0E4
:1004C000C39A1124F0E0E9E66881199278811992C3
:1004D000579B6193579B7193199268811992788108
:1004E0001992579B6193579B71936D817E8177FF22
:1004F00004C07095619508F073950884198417FEFF
:1005000004C01094019408F013946015710518F05C
:100510001694079402C076956795600D711D579BE0
:100520006193579B71931C821D821E821F821886C5
:1005300019862A96C93DC8F2579AC3980F900FBEE4
:10054000FF91EF91DF91CF917F916F911F900F906D
:10055000C2981895529A1895519A18952AE632E041
:10056000DC011696AC014A5A5F4FF901659174910E
:1005700011967C936E932E5F3F4F1A96A417B50782
:10058000A1F720914E00FC01208381EB87B988E818
:1005900083B9089516B808959091D4009D5F6916A7
:1005A00050F0E3EDF0E020E080E0291728F43191ED
:1005B000830F2F5FFACF8FEF08959091D30090387B
:1005C00099F42091D400E5EDF0E0222369F09181C7
:1005D0009E5F29174CF03081381749F0291BE90F2D
:1005E000F11D97FDFA95F1CF80E090E00895CF01DD
:1005F0000895CF93DF93A0D281E0DFDFFC01892B48
:1006000031F1848180930C01858180930D018EE20C
:1006100080930E01928190930F019381909310012A
:100620008093110180E280931201868180931301EF
:100630008781809314018AE38093150180858093DC
:1006400016018185809317011092180105C06DE590
:1006500072E08CE091E078D360E273E084E80DD240
:100660008CE091E038D260E273E080EC06D282E068
:10067000A4DF009771F0FC01C181D0E0BC016E5F86
:100680007F4FAE018CE091E066D3C45FDE4F1882ED
:1006900015C084E092DF009761F0FC0182818F3405
:1006A00029F0803559F461E572E005C064E472E038
:1006B00002C068E372E08CE091E046D38CE091E008
:1006C0000AD26ADF882321F08FE3DF91CF91D7C16F
:1006D000DF91CF910895DF92EF92FF920F931F93D6
:1006E000CF93DF93ADE6B0E00CEF10E02CE031E00B
:1006F000F8018D919D9140815181840F951F8193C7
:1007000091932E173F07A9F757988091FB008F5FB1
:100710008093FB008A30E1F56FEF7FE782E0ADD197
:10072000C0E0D801ED90FD908D01D12CD0E0970173
:10073000232F332722952F702115310521F4D11055
:1007400002C0D33041F4D39480E3820F8A3320F087
:1007500087E3820F01C080E292D184E0EE0CFF1C9F
:100760008A95E1F7DF5FD43011F7CF5FC83039F0F9
:10077000C430B9F660E273E080EC7FD1D2CF109242
:10078000FB0080E1ECEFF0E0DF011D928A95E9F7D4
:10079000DF91CF911F910F91FF90EF90DF9008951F
:1007A000FF920F931F93CF93DF931F92CDB7DEB7C6
:1007B000082FF62E122F861740F4842F49835FD11D
:1007C0000F5F4981F012F9CF15C0681798F460E205
:1007D00073E084E052D1812F52D10150F012FBCF4F
:1007E00060E273E086E00F90DF91CF911F910F914F
:1007F000FF9043C10F90DF91CF911F910F91FF9018
:10080000089589B7877E89BF82E0871528F466201E
:1008100019F077247A940895712C08951F920F92FD
:100820000FB60F9211242F933F934F935F936F93C3
:100830007F938F939F93AF93BF93EF93FF9388B171
:100840002AB1822785FF42C082B790E292279AB9E7
:10085000772041F0822C982F9319292E923210F490
:10086000D0DF34C0382E9AEF980F92BB711005C0BC
:1008700098E098BF99B7986099BF972D913059F03B
:1008800028F0923061F0933091F020C07724739477
:10089000512C412C0AC0420C511C670C04C0251479
:1008A00020F080E1680E711C11C0612C0FC025146E
:1008B00068F4851458F434E0732E8454881982192E
:1008C00083BB80E188BF89B7806189BFFF91EF91C9
:1008D000BF91AF919F918F917F916F915F914F9158
:1008E0003F912F910F900FBE0F901F9018951F9260
:1008F0000F920FB60F9211242F933F934F935F9354
:100900006F937F938F939F93AF93BF93EF93FF93D7
:10091000842D90E095958795482E251418F0282F62
:100920002068422E81E0870D782E8D30C1F08E3008
:1009300061F547FE0DC0262D223058F030E0809141
:10094000D400082E000C990B03962817390709F4D8
:1009500058DF83E0782E89B78F7E89BF19C0862D36
:10096000662019F0813031F008C080E8481629F07F
:1009700048DF03C025E22415D8F3E62D81E0860D7B
:10098000682EF0E0ED52FF4F408283B3805383BB6B
:10099000FF91EF91BF91AF919F918F917F916F9157
:1009A0005F914F913F912F910F900FBE0F901F902D
:1009B00018951F920F920FB60F9211242F933F9309
:1009C0004F935F936F937F938F939F93AF93BF9357
:1009D000EF93FF9316DFFF91EF91BF91AF919F913E
:1009E0008F917F916F915F914F913F912F910F90D8
:1009F0000FBE0F901F90189582E083BF88E188B9E1
:100A0000089580E888B985E083BF0895DC9A25E0E1
:100A10002A95F1F70000DC9828B5222331F096954D
:100A20008795811D911D2150F8CF0197F1F7089509
:100A3000EF92FF921F93CF93DF937B019FE39ABBCB
:100A4000DBB382951D2F107F982F9F70912B9BBB3E
:100A5000C82FC29580E293E0D9DF8C2F8F70812B55
:100A60008BBBC701D3DF80E18ABBD062DBBBDF91E8
:100A7000CF911F91FF90EF900895DD98D9CF60E25C
:100A800073E0D6CF8BE49DE10197F1F700C0000041
:100A90006FEF7FE783E0F1DF80E49FE1B7DF60E2A3
:100AA00073E082E0EADF60E273E088E2E6DF60E2C2
:100AB00073E088E0E2DF6FEF7FE781E0DEDF60E296
:100AC00073E086E0DADF60E273E080E8D6DF60E2C0
:100AD00073E08CE0D2CFCF93DF93EC018991882330
:100AE00011F0CDDFFBCFDF91CF910895CF93DF934E
:100AF000FC018491EF012196882319F0C0DFFE01EB
:100B0000F8CFDF91CF9108950F931F93CF93DF9389
:100B1000EC0160E273E080E4B0DF8E01005C1F4F07
:100B2000FE018491ACDF2196C017D107C9F7DF9190
:100B3000CF911F910F9108956FEF7FE781E09DCFD7
:100B4000CF93DF9300D000D0CDB7DEB780E18ABB72
:100B50008FE28BBB8FE087BB90E798BB83BD8DE4B2
:100B600082BD80E38BBF82E089BF80ED81B978943C
:100B700089DF8AE792E0C8DF9DE3F92E80E888B933
:100B80008FE086BF80E28ABFB69B05C080E285BF4A
:100B900010E00AE08DC080E385BF8091600088236B
:100BA000F9F060E273E080E868DF809160004AE07D
:100BB000BE016F5F7F4F90E0D7D0CE0101968BDFF3
:100BC00081E392E093DF80916000823010F480E254
:100BD00001C085E654DF80E252DF80E250DF03C0CF
:100BE00087E292E083DF8895B69BFDCFCFCF8895D3
:100BF00086B38074892709F02F5F9827519BF7CF20
:100C0000243008F462C0111101C096DF83E192E044
:100C10006DDFEE24E394E10EF9E0FE1508F47CC0EC
:100C200081E3810F2CDF96B39074F2BE51988895C2
:100C300086B38074892798278111F7CF519BF7CF0E
:100C4000B69943C060E273E080E817DF8DE092E080
:100C50004DDF15E080E213DF1150E1F781E0E8128B
:100C600021C060E273E080EC08DF80E092E03EDFCC
:100C7000712CC2DE80EDC82E87E0D82E5198812FCE
:100C80008895172D153008F014E020E24EE2612F10
:100C900087DD812F519BF4CF77FE40C0B2DE77FE17
:100CA00040C0A7DC88E251988895B69B3CC01E2DB9
:100CB00060E273E080E8E1DE06BF12BE85E083BF3C
:100CC000519896B3907420E092CF109260008DE11D
:100CD00092E00CDFF89480E888BD18BC78948DE72A
:100CE00090E03CDCB69B05C08895579BFBCFF3DCBE
:100CF000F9CF8AE0EFE9FFE03197F1F700C000009B
:100D0000B699F0CF8150B1F716B8F89480E888BD55
:100D100083E088BD789432CF83EF84CFB69B0EC03A
:100D2000BDCF0ADFBFCF519BBFCF815009F0BBCFF2
:100D3000809160008F5F8093600020CFE1E0CE1A49
:100D4000D10809F09BCFAACFFB01DC0105900D92E1
:100D50000020E1F70895FB01DC0102C001900D9233
:100D600041505040D8F70895BB27FB015527AA27CB
:100D7000880F991FAA1FA41710F0A41B8395505128
:100D8000B9F7A05DAA3308F0A95DA193009779F7A0
:100D9000B111B1931192CB0100C0DC01FC01672FAE
:100DA00071917723E1F7329704C07C916D93708342
:0E0DB0006291AE17BF07C8F30895F894FFCF05
:00000001FF
